:020000040000FA
:0400040000EF08F011
:06000800010166D91100A0
:10001800D8CF00F0E0CF01F0026E010116D80250EF
:0A00280001C0E0FF00C0D8FF100087
:100040000F01FBEC22F0000102E3D8801200D890EF
:100050001200E9CF03F0EACF04F0FACF05F0FBCFAE
:1000600006F014A73ED09DA03CD09EA03AD09E9012
:10007000CD900201F9504444F92603D00DD017D099
:1000800028D0010181A006D0452A090E456429D057
:10009000442A27D0456A25D0010181B022D06E0EB6
:1000A000436E02016D6B080E476E442A1AD0D89039
:1000B00081B0D8804636472E14D0020EEA6E43C077
:1000C000E9FF46C0EFFF6D2B432A080E476E442A16
:1000D00008D0010181B002D0440603D0446A456AC9
:1000E0002D8A010114A55FD09DA813D09EA811D020
:1000F0009D9813B105D012A503D012892D8009D087
:1001000002EE4BF00A51E926EFCFADFF13810A2B27
:1001100000079DAA48D09EAA46D0356A096AABA2BC
:1001200003D0AB98AB8833D0ABA409D0AE50010E4E
:10013000096E12A72CD03B0EAF6E129728D0426AE0
:10014000AECF07F007BE046B02EE0BF00451E926B8
:1001500007C0EFFF12A704D03B0EAF6E129712D06C
:1001600013A110D002EE4BF00951E926EFCF08F0B1
:100170000750081803E0010E096E04D0092B099BF3
:1001800000679D88096603D02D82042B049B13A170
:100190000AD0095208E013919D9812892D80630EB0
:1001A000AF6EAD6A12879DA687D09EA685D09E961B
:1001B00014AD02D0149D486A4850E844020FF92457
:1001C000F96E0BD016D01DD035D03AD045D04BD0DB
:1001D00050D055D05AD060D063D022C1C9FF212D54
:1001E00002D0010E486E020E216366D0050E486EE5
:1001F00063D0C5BC60D023C1C9FF020E486E2C92EB
:100200005BD0C5BC58D02CB207D014BB05D024C1DC
:10021000C9FF030E486E50D014AB4ED02CB204D0A0
:1002200024C1C9FF2C8248D025C1C9FF149B030EED
:10023000486E42D0C5BC3FD0C584040E486E3CD049
:10024000C00EC614496E496636D0216B226B236BF3
:10025000246B486A9D9630D0C5BC2DD023C1C9FF00
:10026000060E486E29D0C5BC26D0C582070E486E42
:1002700023D0228122C1C9FF080E486E1DD0C5BC03
:100280001AD0C586090E486E17D0C9CF24F1C58A89
:10029000C5880A0E486E10D0C5840B0E486E0CD06F
:1002A000C00EC614496E496606D0216B226B236BC3
:1002B000486A9D9601D02169A1A605D0A196226B1E
:1002C000236B9D96216905C0FAFF06C0FBFF03C0A2
:1002D000E9FF04C0EAFF120014A709D0F2A807D072
:1002E000F2A205D0F292CF68640ECE6ECD8014A536
:1002F00011D0F2A80FD0F2A20DD0F292F29812858E
:10030000356A2DB007D013B105D00D0E0F6102D0A4
:06031000020E0F2712008F
:04032E0000EF02F0EA
:0403560000EF02F0C2
:1004000000011EDE03E30D01F4D90001000100EF3D
:1004100008F01200146A1350146009D09E90B10EB7
:10042000CF6ECD809EA0FED7CD90142AF4D71200B7
:10043000898E126A115012600AD0899E0A0E136EBC
:10044000E9DF898E280E136EE5DF122AF3D7C80E76
:10045000136EE0DFEDD70DEE10F001010351E92638
:10046000EFCF13F00DEE10F0E926EF6A032B400EEC
:100470000361036B13500D011200152C02D0176A93
:10048000000C14C018F0182A1850166201D0186A0F
:100490000D0EEA6E18501324E96EEFCF17F01750C7
:1004A000100A03E0FD0E176EFD0C186A0D0EEA6EC1
:1004B00014501324E96EEF50181A142A14501662BF
:1004C00001D0146A1704196E19521FE0150615BEE3
:1004D00002D0156602D0176A000C0D0EEA6E145099
:1004E0001324E96EEFAE03D0FE0E176EFE0C0D0E58
:1004F000EA6E14501324E96EEF50181A142A14509F
:10050000166201D0146A1906DFD7183C02D01750C2
:1005100012001768FF0C9EAA14D0ABA203D0AB98B0
:10052000AB880FD0ABA402D0AE500BD0899E0DEE9D
:1005300010F00251E926AECFEFFF022B400E026110
:10054000026B0351025D116E11AE02D0400E1126F6
:1005500011522BE00DEE10F00351E926E50EEF628B
:1005600022D0100E136E03C114F011C015F0400E0E
:10057000166E83DF17C091FD0D01915107E0FD0A52
:1005800007E0030A05E0010A06E008D001010DD0EA
:1005900062DF01010AD012680101FF0C898E010E91
:1005A000126E0101010C57DF0101126A000CA6B2A4
:1005B000FED711C0A9FF12C0AAFFA69EA69CA680C6
:1005C000A8501200020E1D6EA69EA69CA68418C0FE
:1005D000A9FF19C0AAFF0DEE00F01BC01CF0EFCF61
:1005E000A8FF550EA76EAA0EA76EA682A6B2FED7CA
:1005F000A680A850EF6209D0020E1D6EEE50A92A07
:10060000A950D8B4AA2A1E8002D01E9002D01C2E57
:10061000E6D71EA002D0D88012001D2EE0D7D890B9
:100620001200899E020E256EA68EA69CA684A68E1A
:1006300020C0F6FF21C0F7FF22C0F8FFA688550EA4
:10064000A76EAA0EA76EA682A6980A000DEE50F01D
:1006500023C024F0EECFF5FF0F00242EFBD7550E5C
:10066000A76EAA0EA76EA682A69420C0F6FF0DEE76
:1006700050F0268023C024F00900F550EE1802E067
:10068000269002D0242EF8D726A004D09281898EFD
:10069000D8801200252ECAD7D8901200A68EA69C0C
:1006A0002250F86E2150F76EC00E2014F66E0DEE3B
:1006B00050F0400E236E0900F5CFEEFF232EFBD73E
:1006C00012003F0E18141F6E500E1F241D6E1D06C3
:1006D0001E6A1F6A1B501F5C1F501B18D8B0800A6F
:1006E00036E61D2A900E1D6219D0500E1D6E93CD58
:1006F00020F094CD21F0226A400E236E92DF0CE3AD
:10070000400E9327000E942393CD20F094CD21F03A
:10071000226AC4DF929102D0D89012000D0EEA6EC8
:100720001EC0E9FFEFCF1CF019501A1003E1030EB1
:10073000186406D00D0EEA6E1DC0E9FF1CC0EFFF65
:100740001E2A182A000E19221A221F2AC3D7D8805F
:1007500012001350176E1250166EC00E1114156E43
:10076000898E175003E1030E166407D0175005E178
:10077000010E155C0A0E16582EE317502CE1F00EF0
:10078000166029D092A10BD015C093FD16C094FD20
:1007900093CD20F094CD21F0226A80DF9291155004
:1007A00093630ED0165094630BD0176609D011C016
:1007B00018F012C019F013C01AF014C01BF081D742
:1007C00093CD20F094CD21F0226A400E236E29DFD4
:1007D000C7E2D8901200F00E136209D011C018F0D1
:1007E00012C019F013C01AF014C01BF0EBD6D88059
:1007F000120092811092899E108001018CDEFF0A06
:100800000D0103E0FE0A07E0C6D010A2C4D0040E1A
:10081000116E0EDEC0D0899E1EDE1DDE100AD8A429
:10082000BAD019DE7F0AD8A4B6D015DE7F0AD8A4C4
:10083000B2D011DE7F0AD8A4AED00DDE0A6E040E4F
:10084000010103250C6E3F0E0C6402D0400E0C5EBD
:100850000DEE10F00C50E926F00EEF140D0108E03B
:10086000100A48E0300A56E0600AD8B485D093D028
:10087000F2DD570A03E0010E116EDADDECDD190A34
:1008800003E0010E116ED4DDE6DD906F909F0AB497
:10089000908F020E010103250C6E3F0E0C6402D0F6
:1008A000400E0C5E0DEE10F00C50E926EFCF0BF071
:1008B0000D010BA00ED00BB207D09051020A09E037
:1008C000020E116EB5DD05D0020E906102D0116EE0
:1008D000AFDDC1DD906F909F0AB6908F0BA408D05A
:1008E000116A126A64DE906103D0030E116EA0DDFE
:1008F000108251D0B0DD0F6E0F9E0AB00F8EABDDAF
:100900000E6E0E9E0AB20E8EA6DD0D6E0D9E0AB400
:100910000D8E41D01DEE00F00C6A040E0C6009D063
:100920009ADDE76E0A32D8A0E69ED8B0E68E0C2A91
:10093000F4D791DD0B6E0C6A040E0C6009D08BDDD0
:10094000E76E0B32D8A0E69ED8B0E68E0C2AF4D71C
:100950000DC011F00EC012F00FC013F0080E146E8F
:10096000F8DE06E3080E0D26000E0E220F2213D02D
:10097000050E116E5DDD0FD092B10CD093CD20F03D
:1009800094CD21F0226A400E236E4BDE03E2050E69
:10099000116E4EDD109010B030D7120054BE09D049
:1009A000D6CF0AF057500A5C585E0AC057F0D8A05C
:1009B000548E1200D6CF0AF055500A5C565E0AC01B
:1009C00055F0D8B012007D0E5626050E0B6E010EA6
:1009D0000C6E00EE4AF054500C140DE1EF06EF3CA3
:1009E00003D0EE50EF06ED50EF50EE50EF1002E165
:1009F0000C505412ED50020EE926000EEA22D89057
:080A00000C360B2EE8D71200A2
:10100000010103D000EC02F001010D0192B303D005
:1010100020EC00F00D010101B5EC23F011EC24F0FF
:1010200007017FEC24F05468556A566AC60ED56EE7
:101030002D6A0101C2EC24F02D862D88D08EF28E0F
:10104000F28C2E6A2F6A306A316A800E416E426ECF
:10105000376E386E3C6E3D6E3E6E3F6E406E356E46
:10106000326E336E346E366E3A6E396E3B6E336A64
:10107000346A366A386A3A6A396A3B6A0400D1903F
:1010800014A703D0326AF292F28888DC93DC2EBE79
:1010900002D06FD82E6E2FBE02D079D82F6E30BE00
:1010A00004D002016ED9306E010131BE02D0C8D920
:1010B000316E32BE02D0F2D9326E33BE02D0B7DA10
:1010C000336E34BE02D050DB346E35BE02D06FDAE0
:1010D000356E36BE02D0DADA366E37BE02D08FDB1E
:1010E000376E38BE02D0A6DB386E39BE05D000019F
:1010F000D6EC15F0396E01013ABE05D0000119ECAD
:1011000013F03A6E01013BBE05D00201C7EC19F0A5
:101110003B6E01013CBE05D000016AEC18F03C6E4C
:1011200001013DBE05D00001A8EC16F03D6E0101A5
:101130003EBE05D0000130EC17F03E6E01013FBE0F
:1011400005D0000126EC1EF03F6E010140BE05D027
:1011500000010DEC20F0406E010141BE03D09FEC78
:1011600010F0416E42BE91D70201A8EC10F0426E21
:101170008CD7F9502E44F92601D004D0010E4A6EC6
:101180004B6A549054A0010CC8EC1CF0000CF950B0
:101190002F44F92601D004D00A0E4C6E4D6A5492A9
:1011A00054A2010C116A020E11603DD003EE00F052
:1011B0001150E926EFCF0EF003EE02F0E9260E50B3
:1011C000EF14106E03EE08F01150E9260E50EF14E4
:1011D0000D6E10500D180F6E010E0C6E0C521BE0B0
:1011E00003EE0AF01150E926EF500F140E6E0C506A
:1011F0000E160EE003EE08F01150E9260C50EF1A1F
:1012000014B306D003EE0EF01150E9260C50EF1285
:10121000D8900C36E3D703EE0AF01150E9260FC040
:10122000EFFF112AC0D73B6A3C6A406A3D6A3E6ABA
:101230002B0EC26EC2B2FED7030EC414186FC3CFFA
:1012400017F1120E175D010E185903E28CEC12F023
:101250000101130EC26E0A6A0B6AC2B2FED7030EF8
:10126000C4140B6EC3CF0AF0810E0A5C010E0B583A
:1012700014E3800E0A5C020E0B580FE214B118D072
:10128000070109A303D00101138F02D00101139FAD
:1012900007010983010114810BD014A109D013AFF8
:1012A00003D00701098302D00701099301011491BA
:1012B000010E0E01486514D03B0EC26E0101C2B290
:1012C000FDD7030EC414186FC3CF17F1185103E1F3
:1012D000680E1765138B185102E1920E1761139B6C
:1012E000010113AB16D02CB409D08AAC07D0899E6B
:1012F0002C84640E0201056F010113872CA409D010
:1013000089AE07D08A9C2C94640E0201086F0101FB
:10131000138913A706D00201052F03D001011397EB
:10132000898E010113A906D00201082F03D0010103
:1013300013998A8C010114A521D081B008D012AF75
:101340000DD00D2B0A0E0D6309D0129F07D00D6B27
:1013500012BF04D00E6702D0010E0E6F0E530EE0C6
:101360000E2B180E0E650AD00E6BF29EF292F288CA
:10137000AB889E9A9D8A9D98F28E128F000C010177
:10138000800C0101F9503044F92601D008D0640ED8
:101390004E6E4F6A5494020154B403D0010C020102
:1013A000FBD701011169020106530EE006070F0E7B
:1013B00006150AE1063B06070F0E061504E0050EAA
:1013C000036F416A068B063B075307E0072F05D0E2
:1013D000050E036F416A010E076F010114A909D0C0
:1013E00013B707D0050E0201036F010E076F416AA4
:1013F000010112AB21D00B800A6A020E02010A60C1
:1014000017D003EE0EF00A50E926EF50D8A40B9047
:1014100003EE16F00A50E926EF50D8A40B9003EE25
:1014200018F00A50E926EF50D8A40B900A2AE5D705
:101430000BA002D00101129B0201000C0201800CE2
:10144000F9503144F92601D005D0E80E506E030E54
:10145000516E549654A6010C12AD1CD0128B03EEA3
:1014600000F01051E926EFCF0AF003EE0EF0E92666
:101470000A50EF1203EE00F01051E926EF1C0A6E3D
:1014800003EE0EF01051E9260A50EF12102B020E57
:101490001061129D1493000C0101800CF95032442C
:1014A000F92600D02DAA010C22EE6DF002EE79F0A3
:1014B0001F0EDF142F6F2F29DECFEEFFE806000A84
:1014C000FBE12D9A326B010E306F2F51306108D045
:1014D00002EE79F03051E926EF50321B302BF5D770
:1014E00002EE79F03051E9263251EF625CD07AC2D7
:1014F00034F1344958D002017AAF30D0050E0101E1
:101500002F612CD002017BAF4ED03F0E7A15040D17
:10151000F3CF34F1070E7B15D890E8300101341376
:10152000040E345F02017B1D700BE83A0F0B0101C2
:10153000356F010E02017B15E83AF00B0101316FA6
:1015400035133451116302D035532DE034C111F1FC
:1015500034C115F135C116F1000E8FDA02017AAFF0
:1015600022D0040E01012F651ED03F0E02017A1514
:101570000101356F7BC234F1345102016B6305D038
:101580000101355102016C1908E00F0E01013463AD
:101590000AD0270E356307D00201EC0E7C15EC0A49
:1015A000D8B4C8EC21F00101000C0101800CF95005
:1015B0003544F92602D007D035D01285D6CF57F062
:1015C000960E586E549E54AE010CF292F2880F455E
:1015D0000A6E0A44060FF924D8B0FA2AF96E960E5C
:1015E0001DD08E0E1BD0860E19D07F0E17D0780E10
:1015F00015D0700E13D0690E11D0610E0FD05A0E97
:101600000DD0520E0BD04A0E09D0430E07D03C0E1F
:1016100005D0340E03D02D0E01D0000ED6CF57F0DA
:10162000586E549E54AE020C12950101800C0201BA
:10163000F9503344F92600D001012DA2010C02011A
:101640000BAF1ED049D90A6E0A50010119E0FF0AFA
:1016500005E102010B6B0101139112D012EE0BF0A8
:1016600004EE00F00251E926E6CFEEFFE950D8B4CF
:1016700004EE00F00A2EF8D7E9CF02F113912D8085
:101680002D922D8C0101000C0101800C3650D8A444
:10169000800C0251031965E004EE00F00351E926C5
:1016A000EFAE5ED004EE00F0E926EF50830A0DE0C5
:1016B000330A0FE0010A22E0030A2FE05F0A3CE050
:1016C000020A47E05B0A4AE04BD00701BFEC10F08A
:1016D00047D044EC10F00AC015F10BC016F11551BB
:1016E0001615FF0A3DE0000EC8D912C00AF013C05B
:1016F0000BF0B1EC14F0139D3F6A32D044EC10F0C3
:101700000AC015F10BC016F115511615FF0A28E095
:10171000010EB3D9139D3F6A23D044EC10F00AC0E8
:1017200015F10BC016F115511615FF0A19E0020E3E
:10173000A4D9139D3F6A14D0E5EC0FF00AC015F14F
:101740000BC016F115511615FF0A0AE0138D3F6AFA
:1017500007D0070174EC20F0010102D0B3EC22F0B5
:10176000032B000C0101800C0201F9503444F926CE
:1017700003D002D02ED038D001012DA4010C2D941D
:1017800002014B390F0B01010F6F0F0E02014B15B8
:101790000101006F010E096F0A6F14A715D0040E26
:1017A000046F596A005159600DD002EE4CF0595047
:1017B000E926EFCF5AF002EE0BF0E9265AC0EFFF10
:1017C000592AF0D72D8217D012B502D012BF03D0FC
:1017D000020C0101F9D7DEEC24F012B5D6D79D88B2
:1017E0002D902DB003D0030C0101FBD712A902D01C
:1017F0001299CBD70F6B2D86000C0101800CF9508C
:101800003744F92600D02DA6010C2D9612EE2BF0B0
:10181000E6CF0AF022EE4BF00AC0DEFF0A060B6AA2
:10182000E6CFDFFFDE500B1A0A2EFAD70B1CDF6E55
:101830002D84800CF9503844F92601D006D0075188
:10184000056303D00851061944E02DA6010C2D961E
:1018500022EE4BF00551E96E050E0625EA6EEFCF3C
:101860000AF00AC0DEFF052B000E0623056705D02F
:10187000020E066302D0056B066B0A060B6A055161
:10188000E96E050E0625EA6EEFCFDFFFDE500B1A7C
:10189000052B000E0623056705D0020E066302D055
:1018A000056B066B0A2EEBD70B1CDF6E0551075D2F
:1018B0000A6E065108590B6E0BAE02D0020E0B26B3
:1018C0000BBE05D0D00E0A5C010E0B58D8A02D8897
:1018D0002D84000C0101800C0BAD14D00BAB0FD08C
:1018E000020E0101046101D0000C0CC20BF0030ECA
:1018F00002010B6403D0100E0B640BD0FF0C060E1C
:101900000B6E07D00BAB03D0040E0B6E02D0020E91
:101910000B6E010104510B6212D00C6A0D6A02EECB
:101920000BF00D50E926EF500C1A0D2A0B500D5CF0
:10193000F6E30C28020102E10B501200FF0C000C30
:10194000176E1438030B1A6E1D9216BE1D821D945D
:1019500016B81D8401011DB014D01DA207D017B008
:1019600005D00F0E1614196E1550186E1DA209D051
:1019700017A007D018C015F019C016F016981DB49E
:1019800016881F0E16161DB019D01A5005E0010A50
:1019900006E0030A0AE011D01686169A31D0169A8C
:1019A000168616A82DD016962BD016341632153260
:1019B0001698D8B01688168A23D012001A5005E05F
:1019C000010A09E0030A10E01AD01686100E14BCB2
:1019D000161A169A15D0169A100E14BC161A1686D8
:1019E00016A80ED016960CD016341632153216984C
:1019F000D8B01688168A080E14BC161A01D0120028
:101A0000D89015361636D89015320751E96E050E66
:101A10000825EA6E040EEF6EA7DB0751E96E050E8E
:101A20000825EA6EB00E1A10EF6E9EDB0751E96EC4
:101A3000050E0825EA6E15C0EFFF96DB0751E96E2B
:101A4000050E0825EA6E16C0EFFF8EDB0551075D17
:101A50001B6E065108591C6E1CAE02D0020E1C26CD
:101A60001CBE06D0E10E1B5C010E1C58D8B02D9890
:101A7000050E0201036F416A12000A6E0F0E161561
:101A8000136E1551126E0F6A020E02010F60DAD149
:101A90000E68010E106E1052D8B4D2D10E2A03EE89
:101AA00000F00F50E926EF1C1014D8B4C6D10F5027
:101AB000400DF3CFD9FFF4CFDAFF100ED926070E71
:101AC000DA22080E0E02F350D926000EDA220EA0FA
:101AD00015D0080ED95E000EDA5ADCCF0BF0DD50BF
:101AE0001C940BBC1C841C960BBE1C861CA602D02E
:101AF0001CA404D0080ED926000EDA22DECF14F082
:101B0000070EDF14156ED9CF1AF0DACF1BF0030ED3
:101B1000D926000EDA22DECF16F0DFCF1DF00F0E31
:101B2000DE14176EDECF18F0DFCF1EF00F0EDE14BE
:101B3000196E1AC0D9FF1BC0DAFFDECF0BF01C9460
:101B40000BBC1C841C960BBE1C86DFCF0CF0DCCFBC
:101B50001FF0DD501F38070B1F6E0B38030B0A6296
:101B600056D01250146253D01350156250D0030E49
:101B70000C144DE01C92010116B91C82020EDFBE4E
:101B80001C1A1F50040A03E0060E1F6209D002014E
:101B90001CB203D01050A51302D0101CA5171C8234
:101BA000020E02010A620ED00AC020F0299029928A
:101BB0001CB229820EC021F00FC022F01050EBECB5
:101BC00014F025D01CB414D01CA612D00EA010D036
:101BD0000AC020F029901CB4298029821CB22992C5
:101BE0000EC021F00FC022F01050EBEC14F00FD01B
:101BF0000AC020F029901CB4298029921CB22982A5
:101C00000EC021F00FC022F01050EBEC14F0030EC8
:101C1000D926000EDA22DFCF0DF0D8900C32D89002
:101C20000C32030E0C147EE01C92010116B91C82CA
:101C3000030E0C14010A05E0030A07E0010A09E09B
:101C40000AD002011CB209D06DD002011CA205D03D
:101C500069D0020102D0020165D00DAE3DD0125014
:101C6000166260D0135017625DD0020E0DBC1C1AB4
:101C70001F50040A03E0060E1F6208D01CB203D0F6
:101C80001050A51302D0101CA5171C821CB414D030
:101C90001CA612D00EA010D00AC020F029901CB4AF
:101CA000298029821CB229920EC021F00FC022F097
:101CB0001050EBEC14F036D00AC020F029901CB480
:101CC000298029921CB229820EC021F00FC022F077
:101CD0001050EBEC14F026D01250146203D01350C5
:101CE000151808E0125018621DD0135019621AD04E
:101CF0001EAE18D002EEAAF00F50E926EFCF11F079
:101D00001CA203D01050111202D0101C111602EEAA
:101D1000AAF00F50E92611C0EFFF03EE16F0E926F6
:101D20001050EF12020ED926000EDA22DFCF0DF08E
:101D3000D8900C32D8900C32030E0C147EE01C921A
:101D4000010116B91C82030E0C14010A05E0030AF6
:101D500007E0010A09E00AD002011CB209D06DD0E7
:101D600002011CA205D069D0020102D0020165D097
:101D70000DAE3DD01250186260D0135019625DD084
:101D8000020E0DBC1C1A1F50040A03E0060E1F624F
:101D900008D01CB203D01050A51302D0101CA517F8
:101DA0001C821CB414D01CA612D00EA010D00AC0E5
:101DB00020F029901CB4298029821CB229920EC0DF
:101DC00021F00FC022F01050EBEC14F036D00AC016
:101DD00020F029901CB4298029921CB229820EC0BF
:101DE00021F00FC022F01050EBEC14F026D012506E
:101DF000146203D01350151808E0125016621DD05B
:101E0000135017621AD01DAE18D002EEACF00F506E
:101E1000E926EFCF11F01CA203D01050111202D00E
:101E2000101C111602EEACF00F50E92611C0EFFFA6
:101E300003EE18F0E9261050EF12D89010362BD68A
:101E40000F2A22D61250010112000751E96E050E29
:101E50000825EA6E0B0EEF6E87D90751E96E050E65
:101E60000825EA6EED0EEF6E7FD90751E96E050E7B
:101E70000825EA6E0B0EEF6E77D90751E96E050E55
:101E80000825EA6E7F0EEF6E6FD90751E96E050ED9
:101E90000825EA6E310EEF6E67D91438E8441F0B3F
:101EA000156E143A1442F80E1416030E131414127D
:101EB000D8901436700E141A1480149ED8901332D1
:101EC000D89013320751E96E050E0825EA6E010E0F
:101ED000EF6E4AD90751E96E050E0825EA6E13C068
:101EE000EFFF42D90751E96E050E0825EA6E14C0CE
:101EF000EFFF3AD90751E96E050E0825EA6E15C0C5
:101F0000EFFF32D90751E96E050E0825EA6EEF6A38
:101F10002BD90751E96E050E0825EA6EEF6A24D920
:101F20000551075D156E06510859166E16AE02D0A2
:101F3000020E162616BE06D0E10E155C010E1658CE
:101F4000D8B02D98050E0201036F416A1200136E7E
:101F50001468010113AD1AD01038E8461F0B1F0B8F
:101F6000176E1238E8461F0B1F0B186E070E10165F
:101F700012160F50116227D01050126224D0146A2A
:101F80001750186220D0010E146E1DD01038030BAC
:101F9000176E1238E840E8423F0B030B186E1750DB
:101FA000186211D00F0E10161214166E1150156E05
:101FB0000F50156208D01050166205D0146A12B87E
:101FC000142A1350141A14501200032B04EE00F0BC
:101FD0000351E926EF500B0A03E00A680B68FF0C77
:101FE000032B04EE00F00351E926EF507F0A03E0D3
:101FF0000A680B68FF0C032B04EE00F00351E9267E
:10200000EF38070B030A03E00A680B68FF0C032B89
:1020100004EE00F00351E926070EEF14010A03E075
:102020000A680B68FF0C032B04EE00F00351E9264D
:10203000EFCF0AF00AAC03D00A680B68FF0CD89007
:102040000A36D8900A36032B04EE00F00351E92635
:10205000EFCF0BF0700E0B1AD8900B32030E0B144F
:102060000A120B3A0B461F0E0B16032B04EE00F060
:102070000351E926EFCF0CF00C3A0C42F80E0C1687
:102080000C500B120A50120004EE00F00351E92626
:10209000EFCF0CF0032B04EE00F00351E926D890AB
:1020A000EF340A6E032B04EE00F00351E926EFCF64
:1020B0000DF004EE00F0E9263F0EEF140B6E0E90CB
:1020C0000DBC0E80030E0C14020A05E0030A0DE09D
:1020D000010A1EE032D00EB003D00A680B68FF0C74
:1020E0000A900DBA0A800B8E28D00EB00BD00DBA14
:1020F00002D00DA804D00DAA05D00DA803D00A68FF
:102100000B68FF0CD8900B320A320B960B8C15D053
:102110000EA003D00A680B68FF0CD8900B320A326D
:102120000BB60AD00AC00FF00BC010F007012ED872
:102130000A680B680101FF0C0B960A50120041500F
:10214000D8A4800C03C205F21387899E0101800C7C
:1021500042500101D8A4800C040E0201086F010155
:1021600013898A9C0101800C072B000E0823076746
:1021700005D0020E086302D0076B086B120009A598
:1021800003D00101106B128D01011200070E101413
:10219000166E0F50156EF80E155C030E1658D8A06B
:1021A000D2D0FC0E155C030E1658D8B0CCD0030E5E
:1021B0000F14146E10B81484116A020E1160BED090
:1021C0001268010E136E1352D8B4B6D0122A1150F1
:1021D000400DF3CFD9FFF4CFDAFF100ED926070E4A
:1021E000DA22080E1202F350D926000EDA22DECFD0
:1021F00017F0DF38030B196E0F0EDE14186E18BCC3
:1022000098D0030E1C6ED890183217321C2EFBD7B4
:10221000186A070E1716DECF1AF01B901ABC1B8027
:10222000030E1A141BE01750146218D009A70AD025
:102230001BA008D0195206E003EE0EF01150E9265B
:102240001350EF1209A90AD01BB008D0196606D0A6
:1022500003EE0EF01150E9261350EF12DE50DECFE0
:1022600017F0DF380F0B196E1B9019B61B80030E89
:1022700019160F0EDE14186E030E1C6ED89018324D
:1022800017321C2EFBD7186A070E17160C0E1A14DD
:102290001BE01750146218D009A70AD01BB008D051
:1022A000195206E003EE16F01150E9261350EF1212
:1022B00009A90AD01BA008D0196606D003EE16F0B3
:1022C0001150E9261350EF12DECF17F0DF380F0B55
:1022D000196E1B9019B61B80030E19160F0EDF1412
:1022E000186E030E1C6ED890183217321C2EFBD7B6
:1022F000186A070E1716300E1A141BE017501462D6
:1023000018D009A70AD01BB008D0195206E003EE76
:1023100018F01150E9261350EF1209A90AD01BA09A
:1023200008D0196606D003EE18F01150E9261350B4
:10233000EF12D890133647D7112A3FD7180E091538
:1023400002E00101128B070112001B6E030EEA6E00
:102350001AC0E9FF1B461B46F9501B44F926EF6AD9
:10236000000E00003BD00A0EEF6E000E37D0140EA8
:10237000EF6E000E33D0230EEF6E000E2FD0320E14
:10238000EF6E000E2BD0410EEF6E000E27D0500ED8
:10239000EF6E000E23D0640EEF6E000E1FD07D0E88
:1023A000EF6E000E1BD0960EEF6E000E17D0C80E0B
:1023B000EF6E000E13D02C0EEF6E010E0FD0900EAC
:1023C000EF6E010E0BD0F40EEF6E010E07D0580E1B
:1023D000EF6E020E03D0200EEF6E030EEC6E1200B5
:1023E0001B6E030EEA6E1AC0E9FF1B461B461B4418
:1023F000060FF924D8B0FA2AF96EE80EEF6E030E34
:102400003BD0DC0EEF6E050E37D0D00EEF6E070E10
:1024100033D0B80EEF6E0B0E2FD0A00EEF6E0F0E56
:102420002BD0880EEF6E130E27D0700EEF6E170EA6
:1024300023D0280EEF6E230E1FD0E00EEF6E2E0E6F
:102440001BD0500EEF6E460E17D0C00EEF6E5D0E15
:1024500013D0300EEF6E750E0FD0A00EEF6E8C0EF7
:102460000BD0100EEF6EA40E07D0800EEF6EBB0ED9
:1024700003D0600EEF6EEA0EEC6E12001B6E030EC0
:10248000EA6E1AC0E9FF1B461B461B44060FF924DF
:10249000D8B0FA2AF96E050EEF6E000E3BD00A0E88
:1024A000EF6E000E37D0140EEF6E000E33D0230EF9
:1024B000EF6E000E2FD0320EEF6E000E2BD0410EBD
:1024C000EF6E000E27D0500EEF6E000E23D0640E7C
:1024D000EF6E000E1FD07D0EEF6E000E1BD0960E1D
:1024E000EF6E000E17D0C80EEF6E000E13D02C0E3C
:1024F000EF6E010E0FD0900EEF6E010E0BD0F40EAA
:10250000EF6E010E07D0580EEF6E020E03D0200EB4
:10251000EF6E030EEC6E120013B561D0070109A136
:102520005ED0F29E900E0C6E010E0D6E0E6A020EC3
:1025300002010E6010D00CC012F00DC013F003EEBB
:1025400008F00E50E926EF50CBEC22F00C2A000EDA
:102550000D220E2AECD70E6A040E0E6010D00CC0AD
:1025600012F00DC013F002EEA6F00E50E926EF5067
:10257000CBEC22F00C2A000E0D220E2AEDD70C2AED
:10258000000E0D220CC012F00DC013F00301075114
:10259000CBEC22F0020E0C26000E0D220201002BC5
:1025A000012302230CC012F00DC013F00051CBEC3C
:1025B00022F00C2A000E0D220CC012F00DC013F0F8
:1025C0000151CBEC22F00C2A000E0D220CC012F0AF
:1025D0000DC013F00251CBEC22F0010113852B0E3C
:1025E000C26E0201C2B2FED7030EC4140101186FFD
:1025F000C3CF17F11D0E175D010E185909E2899E10
:10260000640E176E08D8898E640E176E04D8E7D74B
:10261000D190FF001200186A1750186009D0A192DB
:10262000B10EB36EB180A1A2FED7B190182AF4D733
:102630001200F9503A44F92602D006D02FD05D6A34
:10264000020E5D6057D1010C03EE0EF05D50E926DD
:10265000EF50D8B44DD103EE00F05D50E926EF50B5
:10266000D8B446D15B68010E5C6E5C52D8B440D1E0
:102670005B2A03EE0EF05D50E926EFCF5EF003EE2D
:1026800000F0E926EF505E165C505E14D8B42CD1F1
:1026900003EE0EF05D50E9265C1CEF162DA8020C2F
:1026A0005D50400DF3CFD9FFF4CFDAFF100ED926DD
:1026B000070EDA22080E5B02F350D926000EDA224A
:1026C000DECF60F0616BDFCF61F0DECF0AF0DFCFED
:1026D0000BF0DECF0CF0DECF0DF003EE08F05D5016
:1026E000E9265C50EF146189D8B4619960C01FF18C
:1026F00061C020F10BAE04D0000A6199D8B46189A1
:102700000A38030B04E1010112AB68D0EDD00D389B
:10271000070B64E1010112BB61D003EE04F05D50D0
:10272000E9265C50EF1418E003EE04F05D50E92652
:102730005C1CEF1603EE10F05D50E9265C50EF14C0
:10274000D880D8B4D89004E2000161B9CDD046D089
:10275000000161B943D0C8D003EE14F05D50E92602
:102760005C50EF14000124E103EE10F05D50E92607
:102770005C1CEF1661A913D003EE10F05D50E92642
:102780005C50EF12030E0C14030A28E00DC00EF08B
:102790005BC00FF05DC010F05C50ADD8A5D00DC08F
:1027A0000EF05BC00FF05DC010F05C50A4D89CD060
:1027B00003EE10F05D50E9265C50EF14D880D8B4D9
:1027C000D89003E261B903D009D061B907D003EE14
:1027D00014F05D50E9265C1CEF1686D0030E0C1435
:1027E000010A000107E0030A0AE0010A0BE0030AFC
:1027F0003FE009D0010120A93BD0000104D0010134
:1028000020B936D000010A38030B27E103EE0CF0A3
:102810005D50E926EFCF0EF061AD03D05C500E1A8B
:1028200008D061B902D05C1C0E1661A902D05C50C0
:102830000E1261AF07D05BA003D05C500E1202D025
:102840005C1C0E165C500E146189D8B4619903EEBD
:102850000CF05D50E9260EC0EFFF0AC014F01D9089
:1028600060C015F061C016F05B50A0EC0CF00001E8
:102870001FC160F020C161F0010112BB35D0D890BA
:102880000C32D8900C32030E0C14010A000107E040
:10289000030A08E0010A08E0030A0CE005D061B968
:1028A00003D008D061B906D003EE16F05D50E926DA
:1028B0005C50EF12D8900C32D8900C32030E0C14EE
:1028C000010A07E0030A08E0010A08E0030A0CE035
:1028D00005D061B903D008D061B906D003EE18F075
:1028E0005D50E9265C50EF12D8905C360001BDD6F1
:1028F0005D2AA6D6000C116E0F0E0E14126E0E3845
:10290000070B136E020A02E013662AD0080E1002AB
:10291000F3500F24146E125207E0D89014341A0F9B
:102920001A6E125012DD16D0020E136209D003EE99
:102930001AF0D8901434E9260A0EEE6EEF6A0AD027
:10294000136608D003EE1AF0D8901434E926010E6D
:10295000EE6EEF6A03EE14F01050E9261150EF12FC
:1029600012000A500B14FF0AD8B4120027EE10F020
:10297000116A020E11602ED00F6A010E106E1052F5
:1029800027E0DECF0CF0DFCF0DF00DBE19D0070E23
:102990000D16DECF0EF0129016B912800E38030B12
:1029A0000FE10A500C620CD00B500D6209D02C9034
:1029B00012B02C800C0E11242A6E1050B5EC19F0B8
:1029C000060ED926000EDA220F2AD8901036D7D755
:1029D000112ACFD71200236E29B013D02C9029B220
:1029E0002C80080E22242A6E2350B5EC19F003EE39
:1029F0000EF02250E9262350EF12050E036F416AB4
:102A0000D4D02066D2D021B007D003EE14F02250EB
:102A1000E926231CEF1608D003EE14F02250E92615
:102A2000D8902330FF0AEF1621B027D02C8029B28E
:102A30002C90080E22242A6E2350B5EC19F02C801D
:102A400029B22C90060E22242A6E2350B5EC19F0E0
:102A50002C9029B22C80080E22242A6ED890233480
:102A6000B5EC19F02C9029B22C80060E22242A6E87
:102A7000D8902334B5EC19F098D029B21FD02C90FF
:102A8000080E22242A6E2350B5EC19F02C90060E65
:102A900022242A6E2350B5EC19F02C90080E222423
:102AA0002A6ED8902330B5EC19F02C90060E222413
:102AB0002A6ED8902330B5EC19F077D0D9CF27F013
:102AC000DACF28F02250400DF3CFD9FFF4CFDAFF50
:102AD000130ED926070EDA22080E2102F350D9264A
:102AE000000EDA220F0EDF14256E255006E0050ACF
:102AF00004E00F0A02E0050A27E12C9025B22C80A1
:102B0000080E22242A6E2350B5EC19F02C9025B221
:102B10002C80060E22242A6E2350B5EC19F02C903E
:102B200025B02C80080E22242A6ED8902330B5ECD4
:102B300019F02C9025B02C80060E22242A6ED890F5
:102B40002330B5EC19F02DD02C80080E22242A6EEB
:102B50002350B5EC19F02C80080E22242A6ED89050
:102B60002330B5EC19F0080ED95E000EDA5A5F0E6C
:102B7000DF1417E0060E2114266E080E2202F35011
:102B80002624246E03EE1AF0D8902434E926010E90
:102B9000EE6EEF6A03EE14F02250E926D89023304F
:102BA000EF1227C0D9FF28C0DAFF1200F9503944CC
:102BB000F92602D01AD031D0626B020E6261C7D002
:102BC00003EE0EF06251E926EFCF64F003EE00F061
:102BD000E926EF1C6415D8B4B8D05F68010E636FA6
:102BE0006353D8B4B2D05F2A010C03EE0EF06251E9
:102BF000E926EFCF64F003EE00F0E926EF1C64173E
:102C000063516415D8B49ED003EE0EF06251E926EC
:102C1000631DEF16010112AB3AD000012DA8020C82
:102C20006251400DF3CFD9FFF4CFDAFF110ED92650
:102C3000070EDA22080E5F02F350D926000EDA22C0
:102C4000DDCF0BF00BBC7ED00B38030B7BE1DECF6E
:102C50000CF00D6ADECF0DF003EE08F06251E926AC
:102C60006351EF140D88D8B40D98DFAE04D0000A7C
:102C70000D98D8B40D88100E146E1D900CC015F070
:102C80000DC016F05F50A0EC0CF000015BD000010D
:102C90006251400DF3CFD9FFF4CFDAFF110ED926E0
:102CA000070EDA22080E5F02F350D926000EDA2250
:102CB000DECF65F0DECF66F0DECF67F00F0E671572
:102CC000686F6739070B676F030E66150CE067C006
:102CD00010F068C011F065C012F05FC013F062C060
:102CE00014F0635145D9DCCF0AF0D8906633D89000
:102CF0006633030E66150EE00AAE0CD067C010F006
:102D000068C011F065C012F05FC013F062C014F02B
:102D100063512ED9DE50DCCF0AF0D8906633D890BC
:102D20006633030E66150EE00AAE0CD067C010F0D5
:102D300068C011F065C012F05FC013F062C014F0FB
:102D4000635116D9D89063374BD7622B36D7000C16
:102D5000F9503D44F92602D012D01FD06B6B020E01
:102D60006B617DD003EE16F06B51E926EF5075E0F4
:102D70006969010E6A6F6A5370E0692B010C03EEFA
:102D80000EF06B51E9266A51EF1464E103EE16F080
:102D90006B51E9266A51EF145DE02DA8020C03EE99
:102DA00016F06B51E9266A1DEF166B51400DF3CFFB
:102DB000D9FFF4CFDAFF100ED926070EDA22080E5B
:102DC0006903F350D926000EDA22DCCF0AF0030E95
:102DD000D926000EDA22DECF0BF00C6A3F0EDF148C
:102DE0000C6EDFCF0DF002EEAAF06B51E9266A51AE
:102DF000EF140C88D8B40C980E900ABE0E8003EE27
:102E000000F06B51E9266A51EF140EE00EB00CD0C1
:102E10000A38030B09E103EE0CF06B51E9266A5105
:102E2000EF140C88D8B40C98010112AB07D00D3800
:102E3000030B0F6E0F6602D0100E0D6E0DC014F056
:102E40001D800BC015F00CC016F000016951A0ECFC
:102E50000CF00001D8906A378ED76B2B80D7800C8E
:102E6000F9503E44F92602D012D01FD06D6B020EED
:102E70006D617DD003EE18F06D51E926EF5075E0DD
:102E80006E69010E6C6F6C5370E06E2B010C03EEDB
:102E90000EF06D51E9266C51EF1464E103EE18F069
:102EA0006D51E9266C51EF145DE02DA8020C03EE84
:102EB00018F06D51E9266C1DEF166D51400DF3CFE2
:102EC000D9FFF4CFDAFF100ED926070EDA22080E4A
:102ED0006E03F350D926000EDA22DCCF0AF0050E7D
:102EE000D926000EDA22DECF0BF00C6A3F0EDF147B
:102EF0000C6EDFCF0DF002EEACF06D51E9266C5197
:102F0000EF140C88D8B40C980E900ABE0E8003EE15
:102F100000F06D51E9266C51EF140EE00EB00CD0AC
:102F20000A38030B09E103EE0CF06D51E9266C51F0
:102F3000EF140C88D8B40C98010112AB07D00D38EF
:102F4000030B0F6E0F6602D0100E0D6E0DC014F045
:102F50001D800BC015F00CC016F000016E51A0ECE6
:102F60000CF00001D8906C378ED76D2B80D7800C79
:102F7000156E03EE08F01450E9261550EF14D8B47E
:102F80008DD0080E1402F3501324166E105203E075
:102F9000020E106208D0D89016341A0F1A6E115013
:102FA000A5EC11F01AD0104C03D0030E106208D01B
:102FB000D89016341A0F1A6E1150F0EC11F00DD093
:102FC0001050040A03E0060E106207D0D8901634A1
:102FD0001A0F1A6E11503EEC12F003EE1AF0D89050
:102FE0001634E926EECF18F0EECF19F01050020A91
:102FF0000BE0010A14E0050A12E0060A2DE0010ABE
:1030000036E0050A34E048D01850191008E103EE04
:1030100006F01450E9261550EF12D890120003EE76
:1030200014F01450E9261550EF1436E103EE06F0C3
:103030001450E9261550EF1A03EE1AF0D890163402
:10304000E92618C0EEFF19C0EEFF03EE14F014508D
:10305000E9261550EF1220D01850191008E103EEA0
:1030600006F01450E9261550EF12D890120003EE26
:1030700006F01450E9261550EF1203EE1AF0D8901E
:103080001634E92618C0EEFF19C0EEFF03EE14F067
:103090001450E9261550EF12D88012001050020A81
:1030A0000BE0010A09E0050A07E0060A0BE0010A45
:1030B00009E0050A07E00CD003EE14F01450E926ED
:1030C000151CEF1603EE06F01450E926151CEF163A
:1030D000D8901200F9503C44F92601D005D06F6B0E
:1030E000020E6F61B6D0010C03EE14F06F51E926A9
:1030F000EF50D8B4ACD00B68010E0A6E0A52D8B4A7
:10310000A6D00B2A03EE14F06F51E9260A50EF14F3
:10311000D8B499D06F51400DF3CFD9FFF4CFDAFF77
:10312000100ED926070EDA22080E0B02F350D9260C
:10313000000EDA22DCCF0CF0DCCF0EF0DCCF0DF08D
:103140000D38070B0F6E03EE1AF0080E6F03F350E5
:103150000B24D890E834E926EE06000EEF5A03EE71
:103160001AF0080E6F03F3500B24D890E834E926C8
:10317000EE50EF1068E103EE00F06F51E926EF1C0E
:103180000A144FE00CAC19D0080ED926000EDA2232
:103190000D38F00B0D6E0F0EDF140D26080ED95EE4
:1031A000000EDA5A0FC010F00DC011F00BC012F073
:1031B0006FC013F00A504ED846D00F50020A06E0F6
:1031C0000F50030A03E0060E0F6213D003EE14F053
:1031D0006F51E9260A1CEF160FC010F00F0E0D14E8
:1031E000116E126A0BC013F06FC014F00A50C0DEEB
:1031F00014D00F5205E00F4C03D0040E0F620DD017
:1032000003EE14F06F51E9260A1CEF1603EE06F0E8
:103210006F51E9260A1CEF1616D0010112AB13D02C
:1032200012D003EE14F06F51E9260A1CEF1603EEDC
:1032300004F06F51E9260A50EF1203EE0EF06F51C1
:10324000E9260A50EF12D8900A36000157D76F2BA3
:1032500047D7800C146E03EE06F01350E926196A66
:10326000EFCF18F0125005E01A6ED89018321A2ECF
:10327000FCD7196A030E18161114186212D02C907C
:1032800011B42C80060E13242A6E14506ED82C9084
:1032900011B62C80060E13242A6ED890143465D8EB
:1032A00011D02C9011B02C80060E13242A6E1450CD
:1032B0005CD82C9011B22C80060E13242A6ED89064
:1032C000143453D811380F0B116E080E1302F3503B
:1032D0001224156E03EE14F01350E926141CEF1699
:1032E0001050020A05E0010A1DE0050A1BE033D078
:1032F000D89015341A0F1A6E1150A5EC11F003EE88
:103300001AF0D8901534E926EECF16F0EECF17F06C
:103310001650171020E003EE14F01350E926145055
:10332000EF1219D0D89015341A0F1A6E1150F0EC14
:1033300011F003EE1AF0D8901534E926EECF16F00E
:10334000EECF17F01650171006E003EE14F01350EE
:10335000E9261450EF1203EE1AF0D8901534E9263E
:1033600016C0EEFF17C0EEFF12002B6E030EEA6EC2
:103370002AC0E9FFD8902B50EF14D8A4D8802CA0F5
:1033800003D02B50EF1202D02B1CEF1612000001BD
:10339000F9503B44F92601D0F6D27269010E716FE3
:1033A0007153D8B4F3D2722B746B27EE53F0080E1E
:1033B0007203F350D926000EDA22DFCF73F073BF09
:1033C00074857339070B736F07C370F071517015F3
:1033D0007483D8B4749371510201A51500017481EE
:1033E000D8B47491725115E0010A5FE0030AD8B4B1
:1033F000A8D0010AD8B4F1D0070AD8B43AD1010A4A
:10340000D8B483D1030AD8B4CCD1010AD8B415D228
:103410005FD27E0E0201A617E70EA717060E000167
:10342000736311D07451010A07E0060A05E0040A2B
:1034300007E0060A05E007D00201A681A78703D0AE
:103440000201A68FA789040E0001736118D0745180
:103450000FE0010A0DE0070A0BE0010A09E0050A86
:103460000BE0010A09E0070A07E0010A05E007D0BE
:103470000201A681A78703D00201A68FA789040EA7
:103480000001736325D27451020A07E0050A05E0C2
:10349000040A07E0050A05E01BD20201A681A787FE
:1034A00017D20201A68FA78913D2BD0E0201A6175B
:1034B000DB0EA717060E0001736311D07451010AC9
:1034C00007E0060A05E0040A07E0060A05E007D05F
:1034D0000201A683A78503D00201A68DA78B040E47
:1034E0000001736118D074510FE0010A0DE0070A62
:1034F0000BE0010A09E0050A0BE0010A09E0070AEE
:1035000007E0010A05E007D00201A683A78503D0E2
:103510000201A68DA78B040E00017363D9D17451EB
:10352000020A07E0050A05E0040A07E0050A05E0CB
:10353000CFD10201A683A785CBD10201A68DA78B8F
:10354000C7D1DB0E0201A617BD0EA717060E00019C
:10355000736311D07451010A07E0060A05E0040AFA
:1035600007E0060A05E007D00201A685A78303D07D
:103570000201A68BA78D040E0001736118D074514F
:103580000FE0010A0DE0070A0BE0010A09E0050A55
:103590000BE0010A09E0070A07E0010A05E007D08D
:1035A0000201A685A78303D00201A68BA78D040E76
:1035B000000173638DD17451020A07E0050A05E02A
:1035C000040A07E0050A05E083D10201A685A78366
:1035D0007FD10201A68BA78D7BD1E70E0201A61732
:1035E0007E0EA717060E0001736311D07451010AF5
:1035F00007E0060A05E0040A07E0060A05E007D02E
:103600000201A687A78103D00201A689A78F040E15
:103610000001736118D074510FE0010A0DE0070A30
:103620000BE0010A09E0050A0BE0010A09E0070ABC
:1036300007E0010A05E007D00201A687A78103D0B1
:103640000201A689A78F040E0001736341D1745152
:10365000020A07E0050A05E0040A07E0050A05E09A
:1036600037D10201A687A78133D10201A689A78F8E
:103670002FD17E0E0201A817E70EA917060E000132
:10368000736311D07451010A07E0060A05E0040AC9
:1036900007E0060A05E007D00201A881A98703D048
:1036A0000201A88FA989040E0001736118D074511A
:1036B0000FE0010A0DE0070A0BE0010A09E0050A24
:1036C0000BE0010A09E0070A07E0010A05E007D05C
:1036D0000201A881A98703D00201A88FA989040E3D
:1036E00000017363F5D07451020A07E0050A05E092
:1036F000040A07E0050A05E0EBD00201A881A987CA
:10370000E7D00201A88FA989E3D0BD0E0201A81756
:10371000DB0EA917060E0001736311D07451010A64
:1037200007E0060A05E0040A07E0060A05E007D0FC
:103730000201A883A98503D00201A88DA98B040EDC
:103740000001736118D074510FE0010A0DE0070AFF
:103750000BE0010A09E0050A0BE0010A09E0070A8B
:1037600007E0010A05E007D00201A883A98503D07C
:103770000201A88DA98B040E00017363A9D07451B6
:10378000020A07E0050A05E0040A07E0050A05E069
:103790009FD00201A883A9859BD00201A88DA98B87
:1037A00097D0DB0E0201A817BD0EA917060E000167
:1037B000736311D07451010A07E0060A05E0040A98
:1037C00007E0060A05E007D00201A885A98303D017
:1037D0000201A88BA98D040E0001736118D07451E9
:1037E0000FE0010A0DE0070A0BE0010A09E0050AF3
:1037F0000BE0010A09E0070A07E0010A05E007D02B
:103800000201A885A98303D00201A88BA98D040E0B
:10381000000173635DD07451020A07E0050A05E0F8
:10382000040A07E0050A05E053D00201A885A98330
:103830004FD00201A88BA98D4BD0E70E0201A8172B
:103840007E0EA917060E0001736311D07451010A90
:1038500007E0060A05E0040A07E0060A05E007D0CB
:103860000201A887A98103D00201A889A98F040EAB
:103870000001736118D074510FE0010A0DE0070ACE
:103880000BE0010A09E0050A0BE0010A09E0070A5A
:1038900007E0010A05E007D00201A887A98103D04B
:1038A0000201A889A98F040E0001736311D074511D
:1038B000020A07E0050A05E0040A07E0050A05E038
:1038C00007D00201A887A98103D00201A889A98F86
:1038D0000A6A140E02016AD927C126F12651020193
:1038E000A6190BE00101276B0D6A140E30D9A6C290
:1038F00027F10D6A140E2BD90201010E0A6E150E66
:1039000055D928C126F126510201A7190DE0010160
:10391000286B010E0D6E150E1AD9A7C228F1010EE3
:103920000D6E150E14D90201020E0A6E140E3ED948
:1039300029C126F126510201A8190DE00101296BC8
:10394000020E0D6E140E03D9A8C229F1020E0D6EDF
:10395000140EFDD80201030E0A6E150E27D92AC1D6
:1039600026F126510201A9190DE001012A6B030E6F
:103970000D6E150EECD8A9C22AF1030E0D6E150EB0
:10398000E6D80201010CD89071370AD50201800CEB
:103990000A6A03EE06F00A50E926EFCF0BF003EEB9
:1039A00000F0E926EF1C0B1603EE12F00A50E92690
:1039B000EF500B1A03EE00F00A50E926EFB005D0E5
:1039C0000BA08A980BB08A8807D003EE02F00A5049
:1039D000E926EF9081B8EF8003EE00F00A50E92667
:1039E000EFB205D00BA28A9A0BB28A8A07D003EEF7
:1039F00002F00A50E926EF9281BAEF8203EE00F05E
:103A00000A50E926EFB405D00BA48A940BB48A843B
:103A100007D003EE02F00A50E926EF9481B4EF8458
:103A200003EE00F00A50E926EFB605D00BA68A9601
:103A30000BB68A8607D003EE02F00A50E926EF960D
:103A400081B6EF8603EE00F00A50E926EFB805D004
:103A50000BA889920BB8898207D003EE02F00A50B6
:103A6000E926EF9880B2EF8803EE00F00A50E926CD
:103A7000EFBA05D00BAA89900BBA898007D003EE64
:103A800002F00A50E926EF9A80B0EF8A03EE00F0C8
:103A90000A50E926EFBC05D00BAC89960BBC898691
:103AA00007D003EE02F00A50E926EF9C80B6EF8CB7
:103AB00003EE00F00A50E926EFBE05D00BAE899464
:103AC0000BBE898407D003EE02F00A50E926EF9E70
:103AD00080B4EF8E03EE00F00A50E926EF500B168B
:103AE00003EE02F00A50E9260B50EF1A12000C6A9E
:103AF000040E0C602BD00CB014D001EE27F00C504B
:103B0000E926EF6A0CC00DF0150E21D801EE27F062
:103B10000C50E926EF6A0CC00DF0010E18D8000118
:103B200013D001EE27F00C50E926EF6A0CC00DF01F
:103B3000140E0DD801EE27F00C50E926EF6A0CC0E8
:103B40000DF0000E04D800010C2AD2D712000E6E20
:103B50000101F00E126E13681F0EC5140F6E070ED2
:103B6000C714106E0F66FED71066FCD7060E0D1434
:103B7000226F228D0EC023F1010E216F01EE27F07E
:103B80000D50E926EFCF24F19E969D86C5802153E6
:103B90000CE01206000E135A1250131002E0213DE1
:103BA000F6D70D28146E31D8D4D712000B6E010150
:103BB000F00E0E6E0F681F0EC5140C6E070EC714A4
:103BC0000D6E0C66FED70D66FCD7060E0A14226F2A
:103BD000228D0BC023F1020E216F9E969D86C5801B
:103BE00021530CE00E06000E0F5A0E500F1002E08B
:103BF000213DF6D70A28146E08D8DAD701EE27F04F
:103C00000A50E92624C1EFFF1200020E166E898EBB
:103C1000156A145015600CD0899E0A0E176E0BECB5
:103C200013F0898E280E176E0BEC13F0152AF1D7BE
:103C3000C80E176E0BEC13F0162EE9D79E969D96C4
:103C4000148DC590C66A280EC66E1200F9503F4406
:103C5000F92602D0E5D058D1800E366E2C9E756BB9
:103C6000200E756153D1080E7503F350900F766FD7
:103C7000070E776B772376C0D9FF77C0DAFFDFAE08
:103C800043D1040ED924E16E000EDA20E26E2C9CA2
:103C9000E6CF0BF0E7CF0CF00D6AE7BC0D2A0E90D3
:103CA000E7B80E80DFB802D0E7AE3ED0DFA803D081
:103CB000010113BD05D0DFB835D0010113BD32D0ED
:103CC0000C980BC00FF00CC010F015C111F016C10C
:103CD00012F00D500001A7EC0FF014C00AF00ABE5C
:103CE00021D002EE85F000017551E926EF9C0AB063
:103CF0000CD002EE85F0E926EF9A0AB0EF8A02EEC8
:103D000085F0E926EF900AB0EF8002EE85F075515C
:103D1000E926EF900AB0EF800EA004D002EE85F005
:103D2000E926EF8C000105D002EE85F07551E926F9
:103D3000EF80060ED924E16E000EDA20E26EE6CFA7
:103D40000BF0E7CF0CF00D6AE7BC0D2A0E90E7B838
:103D50000E80DFB602D0E7AE35D0DFA603D001017A
:103D600013BD05D0DFB62CD0010113BD29D00C98AE
:103D70000BC00FF00CC010F015C111F016C112F0FD
:103D80000D500001A7EC0FF014C00AF00ABE18D0C5
:103D900002EE85F000017551E926EFA004D002EE95
:103DA00085F0E926EF8A02EE85F07551E926EF925B
:103DB0000AB0EF820EA004D002EE85F0E926EF8C67
:103DC000000105D002EE85F07551E926EF820E92D2
:103DD000DFBC0E822CBE06D075519AD82C9CD8B070
:103DE0002C8C09D002EE85F07551E926EF9802EE91
:103DF00085F0E926EF9602EE85F07551E926EFB6DB
:103E00002C8E0EB22C9E2CAC7ED0D9CFE1FFDACF17
:103E1000E2FFE4BE05D002EE85F0E926EFB873D0EC
:103E20002DA8010C76C0D9FF77C0DAFFD9CFE1FF0A
:103E3000DACFE2FF070EE4140FE0010A11E0030AF3
:103E400013E0010A15E0070A17E0010A19E0030A66
:103E50001CE0010A1FE022D0010E0A6E0B6A1ED080
:103E6000050E0A6E0B6A1AD00A0E0A6E0B6A16D07D
:103E7000320E0A6E0B6A12D0640E0A6E0B6A0ED0F6
:103E8000F40E0A6E010E0B6E09D0E80E0A6E030ED8
:103E90000B6E04D0880E0A6E130E0B6EE738E846E0
:103EA0001F0B0F0B0C6E0C2A0A500C02F3CF0DF0F7
:103EB000F4CF0EF00F6A0B500C02F3500E26F450A4
:103EC0000F220CAE04D00A500E5E0B500F5A0BAEF0
:103ED00002D00C500F5E0D500E100F1012E003EECA
:103EE0003AF0030E7503F350E9260DC0EEFF0EC045
:103EF000EEFF0FC0EEFF02EE85F07551E926EF8868
:103F000002D07551BBD8020C752BAAD6366A800C2C
:103F10000F6E1190080E0F02F350900FE16E070E16
:103F2000E26AE22202EE85F00F50E926D890E730EF
:103F300006E3EFB002D0EFA206D0118004D0EFA0CC
:103F400002D0EFB21180D890E730030B106E105002
:103F500007E0010A1DE0030A33E0010A41E05BD0FB
:103F600011A013D0EFBC07D011B003D0EFB403D031
:103F700007D0EFB405D0EF86EF84EF9CD880120015
:103F8000EFB649D0EF86D8801200EF96EF9443D079
:103F900011B013D0EFBC07D011B003D0EFB403D0F1
:103FA00007D0EFB405D0EF86EF94EF9CD8801200D5
:103FB000EFB631D0EF86D8801200EF96EF842BD089
:103FC000EFBC07D011B003D0EFB403D024D0EFB4CE
:103FD00022D011A0EF9411B0EF84EF9CD880120092
:103FE00011A017D0EFBA02D0D8901200EFBC07D0C2
:103FF00011B003D0EFB403D007D0EFB405D0EF86F3
:10400000EF84EF9CD8801200EFB605D0EF86D88001
:104010001200EF96EF94D8901200F9504044F92620
:1040200002D006D024D0786B200E786126D0010C07
:1040300002EE85F07851E926EFA81DD003EE3AF0A4
:10404000030E7803F350E926EE06000EEE5AEF5AFF
:1040500003EE3AF0030E7803F350E926EE50EE102B
:10406000EF1009E102EE85F07851E926EF982DA8CE
:10407000020C785103D8782BD7D7800C106E080E1D
:104080001002F350900FE16E070EE26AE222E7AAF7
:1040900012D0020EE126000EE222E6CF11F0126AE3
:1040A000E7CF12F011C013F012C014F0010125EC9B
:1040B0000FF0000118D0020EE126000EE222E6CF3A
:1040C00011F0126A0F0EE714126E1288E7CF13F088
:1040D00013C014F01D8011C015F012C016F0000EB0
:1040E000A0EC0CF00001120009A312000101032B47
:1040F000032B04EE00F00351E9267C0EEF625CD046
:10410000032B04EE00F00351E926EFCF0CF0032B54
:10411000032B04EE00F00351E926EFCF0BF0032B45
:1041200004EE00F00351E926D890EF340A6E0B3408
:104130000B320A320A5002016B6304D00B506C63DD
:1041400001D00BD0010114A107D00F0E0A6204D0D8
:10415000270E0B6201D001D012000101032B032BAB
:10416000FC0E0C14200A0BE0080A09E0040A11E016
:104170004C0A19E0080A17E00C0A1AE01DD00CC01E
:104180000DF00AC00EF00BC00FF017D8010EB3D916
:1041900013D00CC00DF00AC00EF00BC00FF00DD8FC
:1041A000010EA9D909D0F4D8400E0101A4D904D038
:1041B000EFD8400E01019FD9120012EE2BF00E0E27
:1041C000E66EE70EE66E0E0EE66E7C0EE66E0DC037
:1041D000E6FFE66AD8900E360F36D8900E320FC042
:1041E000E6FF0EC0E6FFE66A166A04EE00F0035131
:1041F000E926EFCF14F014C013F013380F0B136E31
:10420000032B04EE00F00351E926EFCF15F015C0A3
:1042100012F0129E14B0128E1790125013100AE171
:10422000040E126E136AE96E070E1324EA6EEFCFC6
:1042300016F01780135003E1050E126412D01350CC
:1042400010E1090E12600DD0060E125E000E135A18
:104250001250E96E070E1324EA6EEFCF16F01780A6
:1042600082D0100E126202D0135205E0110E1262BB
:104270000FD013660DD00C0E125E000E135A1250A2
:10428000E96E070E1324EA6EEFCF16F017806BD09D
:104290001B0E126202D0135205E01C0E12620FD0E8
:1042A00013660DD0150E125E000E135A1250E96EF1
:1042B000070E1324EA6EEFCF16F0178054D06F0E5E
:1042C000126214D0136612D0660E125E000E135ADC
:1042D0001250E96E070E1324EA6EEFCF16F014A108
:1042E00003D0169213BF168217803DD0135003E1FE
:1042F0006F0E126413D0135011E1730E12600ED0C2
:10430000670E125E000E135A900E1224E96E080E0C
:104310001320EA6EEFCF16F0178025D0135002E17C
:1043200012AE12D0135010E112480ED0800E125E61
:10433000000E135A100E1224E96E070E1320EA6EB7
:10434000EFCF16F017800FD013520DE0020E13605E
:104350000AD01306900E1224E96E070E1320EA6E9F
:10436000EFCF16F01780149216BE148214C0E6FF29
:1043700015C0E6FF7F0E1614E66EE66AE66A17A021
:1043800005D0050E0201036F416A0101138312007B
:104390001190010114A70ED00C0E02017C150C0A1D
:1043A000D8A41200030E7C15106E7DC20FF07EC2E1
:1043B0000DF0010114A51DD004EE00F00351E92613
:1043C000EFCF10F0032B04EE00F00351E926EFCFFE
:1043D0000FF00F9E10B00F8E032B04EE00F0035170
:1043E000E926EFCF0DF00D9E10B20D8E10380F0B99
:1043F000106E10502FE1200E0F602CD0100E0F62A7
:1044000002D0105205E0110E0F620ED010660CD0D3
:104410000C0E0F5E000E105A0F50E96E070E10249E
:10442000EA6E0DC0EFFF58D01B0E0F6202D0105283
:1044300005E01C0E0F6250D010664ED0150E0F5EB8
:10444000000E105A0F50E96E070E1024EA6E0DC0D0
:10445000EFFF42D06F0E0F6213D0106611D0660EC0
:104460000F5E000E105A0F50E96E070E1024EA6E10
:10447000800E0D10EF6E139F0DB2138F11802CD094
:10448000105002E10FAE14D0106612D0800E0F5EF5
:10449000000E105A100E0F24E96E070E1020EA6E5F
:1044A0000DC0EFFF100E0F26000E1022118014D049
:1044B000105211E0020E10600ED01006900E0F2464
:1044C000E96E070E1020EA6E0DC0EFFF900E0F266A
:1044D000000E102201D012000FC012F010C013F015
:1044E0000D5059D811A002D09CD94CDA050E02010A
:1044F000036F416A12000D6E0751E96E050E082523
:10450000EA6E040EEF6EB4EC10F00751E96E050E82
:104510000825EA6EB40EEF6EB4EC10F00751E96EA8
:10452000050E0825EA6E6F0EEF6EB4EC10F0075121
:10453000E96E050E0825EA6E0DC0EFFFB4EC10F031
:104540000551075D0E6E065108590F6E0FAE02D071
:10455000020E0F260FBE06D0E10E0E5C010E0F58A4
:10456000D8B02D981200032B04EE00F00351E92679
:104570006F0EEF6204D013A302D01393376A1200B8
:10458000A6B2FED715C0A9FF16C0AAFFA69EA69C7C
:10459000A680A8501200146E12C015F013C016F0B9
:1045A000EFDF14181CE0A6B2FED714C0A8FF12C09B
:1045B000A9FF13C0AAFFA69EA69CA684F29E550E34
:1045C000A76EAA0EA76EA682F28EA69412C015F050
:1045D00013C016F0D5DF141802E0D8901200D8806E
:1045E00012007FCFF6FF7FCFF7FFF86AA68EA69C5A
:1045F0000800F5501200F00ED36EC00E9B6E100E28
:10460000386F020E396F040E3A6F110EC26EC16A16
:10461000BE0EC06E800E806E2F0E926E400E816EAA
:10462000BF0E936E616A826AFC0E946E270EC86E8E
:10463000280EC66EC56ACB6AC76A200EAC6E900E95
:10464000AB6E100EB86E3B0EAF6EF26AF16AF06A96
:104650009D6AA06A9F6AA26AD59ED66A340ECD6E04
:104660009E909D90CE0EBA6EBA94300EB16E2B0E07
:10467000C26E0101C2B2FED7030EC414186FC3CFBD
:1046800017F1220E175D010E18590BE2899E640E78
:10469000176E0BEC13F0898E640E176E0BEC13F093
:1046A000E6D7D08EF28EF28C000177EC1DF0F29EF0
:1046B000F29C0FEE37F00101ED6AEA50FDE1E9509E
:1046C000FBE1EF6AA68EA69CF66AF76AF86A0EEE20
:1046D00000F0400E0C6E0900F552F5CFEEFF0C2EE7
:1046E000FAD70C6A10800EEE00F00C50E926EFCFDE
:1046F0000DF0AAD90E6E0D500E6210900C2A070E06
:104700000C64F1D710B01CD00C6A080E0C600BD0F2
:104710000C509AD90D6E0EEE00F00C50E9260DC02B
:10472000EFFF0C2AF2D75AD90BE2899E960E176E2C
:104730000BEC13F0898E960E176E0BEC13F0F3D77B
:104740000D019283130EC26E0101C2B2FDD7030E9A
:10475000C4140B6EC3CF0AF0010E0A5C030E0B5893
:1047600002E3D8801200D890120007EE00F00A6A27
:104770000B6A0AC015F00BC016F002DFEE6E0A2AB3
:10478000000E0B229C0E0A5C010E0B58F2E399C836
:1047900000F29AC801F29BC802F23F0E070104150D
:1047A00002016C6F05C76BF2A68EA69CF66AF76ACB
:1047B000200EF86E0EEE40F0080E126E0900F5CFD6
:1047C000EEFF122EFBD745CE48FE130EC26E01013E
:1047D000C2B2FED7030EC414116EC3CF10F01499E9
:1047E00014971495200E105C010E115802E21485E6
:1047F00017D0220E105C010E115807E3800E105CDA
:10480000010E115802E214870BD0820E105C010ECB
:10481000115806E3800E105C020E1158D8A01489BE
:10482000120027EE12F0156A020E156027D0010E55
:10483000146E03EE12F01550E926EF6A03EE00F055
:10484000E926EF6ADFAC07D003EE00F01550E92649
:104850001450EF1209D0DCAE06D003EE12F0155062
:10486000E9261450EF12DD50D8901436080ED926E0
:10487000000EDA221466E6D7152AD6D7200E926EDD
:10488000830E936EDC0E946E156A03EE00F01550E5
:10489000E926EFAA9290EFBA928003EE00F0E926A3
:1048A000EFA89292EFB8928203EE00F0E926EFAE05
:1048B0009294EFBE928403EE00F0E926EFAC92965C
:1048C000EFBC928603EE00F0E926EFA09398EFB0DC
:1048D000938803EE00F0E926EFA2939AEFB2938A51
:1048E00003EE00F0E926EFA49394EFB4938403EE73
:1048F00000F0E926EFA69396EFB69386120009A181
:1049000040D027EE11F00B6A020E0B603AD0010E78
:104910000D6E0C6ADFCF0EF0020ED926000EDA22E1
:10492000DFCF0FF00F38070B0F6E0EBC04D0040A58
:1049300002E00D500C12D8900D36060ED926000E4E
:10494000DA220D66E7D7900E0B24E96E080EEA6AAC
:10495000EA22EFCF0AF003EE08F00B50E9260C50E4
:104960000A14EF6E03EE00F00B50E926EF1C0A6EFE
:1049700003EE0EF00B50E9260C500A14EF6E0B2AD2
:10498000C3D71200016B126A100E12600CD0080E11
:104990001202F350100FD96E070EDA6ADA22DF50D6
:1049A0000127122AF1D7040E02016B03F350010113
:1049B00001273F0E011701C106F712000A6A0151D3
:1049C0000A600BD0A192B368B26AB180A1A2FED7EF
:1049D000B19012B502D00A2AF2D71200020E116E5F
:1049E000A68EA69CA684A68EF66AF76AF86AA688A2
:1049F000550EA76EAA0EA76EA682A6980A000EEE06
:104A000000F0400E126EEECFF5FF0F00122EFBD716
:104A1000550EA76EAA0EA76EA682A694F66A0EEE93
:104A200000F01380400E126E0900F550EE1802E0FF
:104A3000139002D0122EF8D713A002D0D880120003
:104A4000112ED0D7D8901200116E5C0FF66E4A0E60
:104A5000F76AF722F86A0800F550120000EF02F03A
:044A600000EF08F06B
:0200000400F00A
:1000000013571900270F00E0009F000000000000B8
:100010000020430000000000012043000000000019
:100020000220430000000000032043000000000005
:1000300004204300000000000520430000000000F1
:1000400006204300000000000720430000000000DD
:100050000800030000000000090003000000000089
:100060000A000300000000000B0003000000000075
:100070000C000300000000000D0003000000000061
:100080000E000300000000000F000300000000004D
:100090000000000000000000000000000000000060
:1000A0000000000000000000000000000000000050
:1000B0000000000000000000000000000000000040
:1000C0000000000000000000000000000000000030
:1000D0000000000000000000000000000000000020
:1000E0000000000000000000000000000000000010
:1000F0000000000000000000000000000000000000
:1001000000000000000000000000000000000000EF
:1001100000000000000000000000000000000000DF
:1001200000000000000000000000000000000000CF
:1001300000000000000000000000000000000000BF
:1001400000000000000000000000000000000000AF
:10015000000000000000000000000000000000009F
:10016000000000000000000000000000000000008F
:10017000000000000000000000000000000000007F
:10018000000000000000000000000000000000006F
:0C01900000000000000000000000000063
:020000040000FA
:0400000000EF02F01B
:020000040030CA
:0E000000FF280008FF8181FF0FC00FE00F40B6
:00000001FF
